:1000000000308A00982A00000A108A100A1182071C
:100010005034493443342034313436344634363461
:10002000323438344134203447345034533420345B
:1000300048346F34723461342F3446346534633459
:1000400068346134203470346F34723420342E3488
:1000500052344134443449344F34563441344C34AE
:100060004C34413444344F344C34493444342E34C9
:1000700043344F344D340D340A3400340A108A109E
:100080000A11820756346534723473346934F33498
:100090006E34203456342E34313420344A3475349E
:1000A0006E3469346F34203464346534203432342F
:1000B00030343034373420342834AE3429342C34BE
:1000C000203474346F3464346F34733420346C34BB
:1000D0006F3473342034643465347234653463347B
:1000E00068346F3473342034723465347334653457
:1000F00072347634613464346F3473342E340D3496
:100100000A3400340A108A100A1182073134373455
:100110002D347334653470342D3430343734003436
:100120003C08073C031899280130C0000830BC0285
:100130009A28C0013C08033C0318A3280130BF00E3
:100140000430BC02A428BF013C08013C0318AD28C0
:100150000130BE000230BC02AE28BE013C0BB32809
:100160000130BD00B428BD01C008031DBC288316A2
:10017000861383128613C02883168613831286176C
:10018000BF08031DC8288316061383120613CC2844
:100190008316061383120617BE08031DD428831680
:1001A000861283128612D828831686128312861628
:1001B000BD08031DE0288316061283120612E428E8
:1001C00083160612831206163B08073C031DF4280B
:1001D0008316051183120515831685108312851465
:1001E00083160510831205143B08063C031D0429E1
:1001F0008316051183120515831685108312851445
:1002000083160510831205103B08053C031D1429B5
:100210008316051183120515831685108312851028
:1002200083160510831205143B08043C031D242982
:100230008316051183120515831685108312851008
:1002400083160510831205103B08033C031D342957
:1002500083160511831205118316851083128514E8
:1002600083160510831205143B08023C031D442924
:1002700083160511831205118316851083128514C8
:1002800083160510831205103B0B522983160511A6
:1002900083120511831685108312851083160510AD
:1002A00083120514BB08031D6129831605118312EF
:1002B000051183168510831285108316051083128D
:1002C0000510831685118312851100008316851190
:1002D0008312851500343B308400000803197F2900
:1002E0000130F800F701F70B7329F80B72294A3037
:1002F000F700F70B792900000000800B702900340B
:100300008C1E80291808A0001A08F800A01C8A2951
:100310001812181600000034BA01BB01BB08031DF7
:10032000BA2980217808BA003A08473C031DB92948
:1003300080217808BA003A08503C031DB929802171
:100340007808BA003A08523C031DB9298021780880
:10035000BA003A084D3C031DB92980217808BA003B
:100360003A08433C031DB92980217808BA000130BE
:10037000BB008E29872BBA01BB013A0BC029C829C3
:10038000802178082C3C031DC7290130BA00BD2903
:100390000034BA01BB01BB08031DF729802178088E
:1003A000BA003A08473C031DF62980217808BA00B4
:1003B0003A08503C031DF62980217808BA003A0813
:1003C000473C031DF62980217808BA003A08473CCB
:1003D000031DF62980217808BA003A08413C031D24
:1003E000F62980217808BA000130BB00CB29A52B63
:1003F000F701F801410803104218F707F70CF80C51
:10040000C218F707F70CF80C4219F707F70CF80CAD
:10041000C219F707F70CF80C421AF707F70CF80C9B
:10042000C21AF707F70CF80C421BF707F70CF80C89
:10043000C21BF707F70CF80C00344308F80142021E
:100440000318252A4208F700312AF7010830C400B2
:10045000C20DF70D430877020318F700F80DC40B1F
:10046000282A00343E08C2000A30C3001D22780842
:10047000BE003E08F80000343F08C2000A30C30046
:100480001D227808C0004008C1000A30C200F821CF
:100490007808C0004008BF023F08F8000034400858
:1004A000F700C01B572A411D642A20305C2AF70937
:1004B000F70A7708C0002D30F80078080C1E5E2A75
:1004C00099001030C11DC1004008C2006430C30053
:1004D0001D227708C00078083030031D762A4118A5
:1004E0007D2AC1197D2A411A2030782AC111411272
:1004F000F80778080C1E7A2A99004008C2000A30D2
:10050000C3001D227708C00078083030031D8C2AF4
:10051000C119912A411A2030F80778080C1E8E2A3A
:1005200099003030C00740080C1E942A990000340E
:1005300084011F30830507309F000C30831699001B
:1005400022309800903083129800A0010730BB0041
:100550000830BC0090200630BB000830BC00902062
:100560000530BB000830BC0090200430BB000830D0
:10057000BC0090200330BB000830BC00902002304B
:10058000BB000830BC0090200130BB000830BC002C
:100590009020BB010830BC0090200630BA00FA3031
:1005A000BB006B21BA0BCF2A0730BB00BC009020E8
:1005B0000630BB000830BC0090200530BB00013085
:1005C000BC0090200430BB000230BC0090200330FF
:1005D000BB00BC0090200230BB000430BC00902067
:1005E0000130BB000530BC009020BB010630BC00D0
:1005F00090200630BA00FA30BB006B21BA0BFB2A00
:100600000730BB00BC0190200630BB000F30BC009F
:1006100090200530BB000A30BC0090200430BB00A5
:100620000B30BC0090200330BB000C30BC0090208D
:100630000230BB000D30BC0090200130BB000E30FA
:10064000BC009020BB010F30BC0090200630BA00E7
:10065000FA30BB006B21BA0B282B0D300C1E2E2B51
:1006600099000430BA000A300C1E342B9900BA0BE2
:10067000332BBA013A080420BA0AF70077080C1E97
:100680003F2B99001F303A02031D3A2B0330BB0069
:1006900057300C1E492B9900BB0B482B1F30BC0058
:1006A0003C080420BC0AF70077080C1E552B990063
:1006B00035303C02031D502BBA013A083E20BA0ADD
:1006C000F70077080C1E622B99003F303A02031D99
:1006D0005D2BBA013A088220BA0AF70077080C1E8F
:1006E0006F2B990009303A02031D6A2B0D300C1E46
:1006F000772B99000430BA000A300C1E7D2B99002C
:10070000BA0B7C2B83160512831205168C29BB218C
:1007100080217808AD00BB21BB21BB21BB21BB21BF
:10072000BB21BB2180217808A70080217808A80080
:1007300080217808A90080217808AA008021780803
:10074000AB0080217808AC00C92980217808A1007D
:1007500080217808A20080217808A30080217808F1
:10076000A40080217808A50080217808A600BB217C
:10077000BB21BB21BB21BB21BB2180217808B80054
:1007800080217808B90030302102BB00C1000A3056
:10079000C200F821303022027807A1003030230255
:1007A000BB00C1000A30C200F821303024027807B3
:1007B000A30030302502BB00C1000A30C200F8217E
:1007C000303026027807A50030302702BB00C10078
:1007D0000A30C200F821303028027807A7003030F4
:1007E0002902BB00C1000A30C200F82130302A02C1
:1007F0007807A90030302B02BB00C1000A30C200CC
:10080000F82130302C027807AB0030303802BB00C2
:10081000C1000A30C200F821303039027807B80030
:10082000831606140030831206180130013C031DA4
:100830005F2C0730BB003108BC0090200630BB00A5
:100840003808BC0090202708BE0032227808BA0081
:100850000530BB007808BC0090202708BF003C2270
:100860007808BA000430BB007808BC009020290842
:10087000BE0032227808BA000330BB007808BC0002
:1008800090202908BF003C227808BA000230BB0043
:100890007808BC0090202B08BE0032227808BA00ED
:1008A0000130BB007808BC0090202B08BF003C2220
:1008B0007808BA00BB017808BC009020AC2C2D0849
:1008C000413C031D662C0130AD00672CAD010730A3
:1008D000BB002D08BC0090200630BB002E08BC00D9
:1008E00090202108BE0032227808BA000530BB00F3
:1008F0007808BC0090202108BF003C227808BA008C
:100900000430BB007808BC0090202308BE003222CF
:100910007808BA000330BB007808BC009020230898
:10092000BF003C227808BA000230BB007808BC0047
:1009300090202508BE0032227808BA000130BB00A2
:100940007808BC0090202508BF003C227808BA0037
:10095000BB017808BC0090202108BE003222780834
:10096000BA002108BF003C227808BB002308BE0063
:1009700032227808BC002308BF003C227808BD0062
:100980002508BE0032227808BE002508BF003C22A0
:100990007808BF0024300C1ECB2C99003A08C00008
:1009A0001830C1004F223B08C0001830C1004F2250
:1009B0003A300C1ED92C99003C08C0001830C100F8
:1009C0004F223D08C0001830C1004F223A300C1EA3
:1009D000E72C99003E08C0001830C1004F223F08A4
:1009E000C0001830C1004F222C300C1EF52C99008D
:1009F0002708BE0032227808BA002708BF003C2230
:100A00007808BB002908BE0032227808BC002908FB
:100A1000BF003C227808BD002B08BE0032227808B7
:100A2000BE002B08BF003C227808BF003A08C00077
:100A30001830C1004F223B08C0001830C1004F22BF
:100A40002F300C1E212D99003C08C0001830C10029
:100A50004F223D08C0001830C1004F222F300C1E1D
:100A60002F2D990032300C1E332D990030300C1E82
:100A7000372D99003E08C0001830C1004F223F08B2
:100A8000C0001830C1004F222C300C1E452D99009B
:100A90002E08C0001830C1004F222C300C1E4E2DE5
:100AA00099003108C0001830C1004F220D300C1ED3
:100AB000572D99000A300C1E5B2D9900862B630080
:104200004A006100760069006500720020005200DB
:104210006F0064007200ED006700750065007A00B1
:104220002C0020007700770077002E0072006100DC
:10423000640069006F00760061006C006C00610032
:1042400064006F006C00690064002E0063006F0062
:104250006D002000520065006C006F006A002000B5
:104260004700500053002000560041004C00490018
:1042700044004F002000480041005300540041001A
:10428000200045004C0020004100D1004F002000DC
:104290003200300039003900200054006F00640003
:1042A0006F00730020006C006F007300200064003A
:1042B000650072006500630068006F0073002000F5
:1042C0007200650073006500720076006100640092
:1042D0006F00730020002800AE00290020004A0073
:1042E00075006E0069006F00200032003000300061
:1042F000370020002A0028005F0029002A00000063
:02400E00013F70
:00000001FF
